:040000008A15002835
:0E000600F201F101F001F801F30100300800F1
:100014007B15FB1F14280130F300F201F101F001FC
:08002400FA0DF20CFF30080098
:08002C00FA1FF2130030080076
:10003400FB14FB1F2428FF30F300F200F100F00052
:08004400FA0DF20CFF30080078
:0E004C00533083120313FD00FD0B2A28080019
:10005A00A0017208031D42287108F2007008F1001D
:10006A00F001A0157208031D42287108F200F1017F
:10007A00A01120167208031950282008F302031D44
:10008A00031C54280310F21B5828F00DF10DF20D31
:10009A00F30B482854280130FC0003205B28023067
:0E00AA00FC000A205B280430FC001620080031
:1000B8007C189228FC1863287C19B1285C28A001B8
:1000C8007208031D83287108F2007008F10078088F
:1000D800F000F801A0157208031D83287108F200CA
:1000E8007008F100F001A01120167208031D832882
:1000F8007108F200F101A01572080319A52820085B
:10010800F302031D031CA9280310F21B9228F80D03
:10011800F00DF10DF20DF30B8928A9287B1B701C3B
:10012800AD28F81FAD28F00A0319F10A0319F20ADD
:10013800031DAD28F20CF10CF00CF30A0319B128D9
:10014800AD280130FC000320B4280230FC000A204E
:10015800B4280430FC001620B4280830FC001A200B
:04016800000008008B
:10016C00243083120313FC00B530FD00FD0BBC28BA
:0A017C00FC0BBC2800000000080086
:0C01860000000000000000000000080065
:100192007B14FB1FD428F201FA1FFF30F200F1009A
:0A01A200F000FA0DF20CFF30080027
:1001AC0083160313AD1BDD2883128611DF288312FF
:1001BC00861583162D1BE52883120611E72883125A
:1001CC0006158316AD1AED2883128610EF288312BC
:1001DC00861483162D1AF52883120610F72883121D
:1001EC0006143918FB288515FC2885118514C320A5
:1001FC0085108316AD1905298312861107298312E0
:10020C00861583162D190D29831206110F298312B9
:10021C0006158316AD18152983128610172983121B
:10022C00861483162D181D29831206101F2983127C
:10023C000614391823298515242985118514C32002
:0E024C008510391C2B29B6202C2926200800ED
:06025A00FB15FF30080057
:100260008312031372087606A000F801F9017308DF
:100270007702031C53297708FD007308F7007D08F7
:10028000F3007608FD007208F6007D08F20075089C
:10029000FD007108F5007D08F1007408FD0070088C
:1002A000F4007D08F00077080319CC297208FA00E1
:1002B000F217F61777087302F7000319862908303A
:1002C0007702031C7C29F7007408F9007508F40014
:1002D0007608F500F60108307702031C7C29F70048
:1002E0007408F9007508F400F50108307702031C62
:1002F0007C297A08F200CC29770803198629031093
:10030000F60CF50CF40CF90CF70B7F29A01F9329C0
:10031000F909F409F509F609F90A0319F40A0319A8
:10032000F50A0319F60A7908F80774080318740F18
:10033000F00775080318750FF10776080318760F94
:10034000F207A01BAC29031CBC29F20CF10CF00C29
:10035000F80CF30FBC29C8290318C029F809F009C3
:10036000F109F209F80A0319F00A0319F10A03194D
:10037000F20A8030FA06C4290130FC005C20CE2944
:100380000230FC005C20CE290430FC002D20CE2958
:100390000830FC001A20CE290030FC0000000800C4
:1003A00083120313FB017308031D77080319272A1F
:1003B00072087606FA007708F3077E30031CE429FA
:1003C000F30203182A2AE729F302031C2D2A7208D4
:1003D000F8007108FC007008FD00F817F61703100C
:1003E000F201F101F0011830A0007D1C012A74080F
:1003F000F00775080318750FF10776080318760FD4
:10040000F207F20CF10CF00CF80CFC0CFD0C0310D4
:10041000A00BF529F21B112AF80DF00DF10DF20DCC
:10042000F3037B1B701C232AF81F232AF00A0319ED
:10043000F10A0319F20A031D232AF20CF10CF00C45
:10044000F30A03192A2AFA1FF21300302F2A013067
:1004500003202F2A02301A202F2A04300A200000FD
:02046000080092
:10046200831203137408003A031D4C2A7508003ADC
:10047200031D4C2A7608003A031D4C2A7708003ADD
:10048200031D4C2AFF30F000FF30F1007F30F200F4
:10049200FF30F300E72A8312031377080319DB2ADC
:1004A20073080319DE2A720876068039FA00F217F9
:1004B200F617A0017208F8007108FC007008FD0030
:1004C2007408FD027508031C750FFC027608031CF4
:1004D200760FF802F801FC01FD01031C772A0310D4
:1004E200F20CF10CF00CF80C0130A0007708F302CA
:1004F200031C812A7E302007F3070318E12A862A8B
:100502007E302007F307031CE42A1830FA07FD0D9A
:10051200FC0DF80DF00DF10DF20DA00D7408F002B6
:100522007508031C750FF1027608031C760FF202A0
:10053200760DA004201C9F2A7D14AA2A7408F007B5
:1005420075080318750FF10776080318760AF20783
:100552007D10FA031F307A05031D882A7B1B7D1C40
:10056200D12A0310F00DF10DF20DA00D7408F00266
:100572007508031C750FF1027608031C760FF20250
:10058200760D20040139FD070318FC0A0319F80A45
:10059200031DD12AF80CFC0CFD0CF30A0319E12A05
:1005A200FA1FF8137808F2007C08F1007D08F000C9
:1005B2000030E62A01302D21E62A02300320E62A05
:0E05C20004301A20E62A08300A200000080043
:1005D000831203137008F8007108F000F101F201B2
:1005E000F301FB01FC019630F300FA01F01FFE2A33
:1005F000F809F009F80A0319F00AFA177008F1006F
:0C0600007808F000F801F2012D2008003D
:0C060C00831203138030F6063021080032
:1006180083120313FB0173080319492B7208FA00AC
:10062800F2178E30F302F31F4C2BF309F30A08304C
:100638007302031C2F2BF300F10D7208F100F20175
:1006480008307302031C2F2BF300F10DF10173081E
:10065800031D0310372B73080319372B0310F20CF3
:10066800F10CF30B322B7B1B711C412B031C412B10
:10067800F10A0319F20AF21B582BFA1F5B2BF20935
:10068800F109F10A0319F20A5B2BF201F1015B2B64
:100698007B14FB1F5E2BF201FA1F5E2BFF30F2006A
:1006A800F100FA0DF20C5E2B0130FC00602B0030DB
:1006B800FC00602BFF30FC00FC080319642BC920E8
:0A06C8007108F0007208F10008004C
:1006D20083120313FA017308031D7A147708031DAA
:1006E200FA147A080319B52B033A0319802B7A18E6
:1006F2007D2BF61FB32BB12BF21FB12BB32B72083C
:100702008039FA00F21376088039F6137A06031953
:100712008E2B7A080319B12BB32B770873020319B6
:10072200952B031CA92BAD2B7608720203199C2B67
:10073200031CA92BAD2B750871020319A32B031CF3
:10074200A92BAD2B740870020319B52B0318AD2B1E
:10075200FA080319B32BB12BFA080319B12BB32BE7
:10076200031408000310080003140315080008000E
:1007720083120313391083162C08AD00D6203914C6
:0207820008006D
:1007840083120313EA016A08690784000008031945
:10079400D42B6A086907840000088316AC00B923C7
:0607A400EA0AC52B080063
:1007AA00831203136908F2007208F000F20A700853
:1007BA00840000080319E22BD92B69087202F000A1
:0C07CA000130F002F101031CF1030800F3
:1007D600831203136D08EF006E08003C031CF82B10
:1007E6000730F4000030F5000F2C6E08163C031895
:1007F600012C1730F2000030F3000B2C6E08013E7E
:10080600F000F1010318F10A7008F2007108F30014
:100816007208F4007308F50074088316A6007508BC
:10082600A700A001A101F401F501F601F701831269
:100836006908F0006A08F1006B08F2006C08F30022
:100846006923013003180030F00070080319382CB2
:100856006D0884002D308000ED0A0030E906003076
:10086600EA068030EB060030EC066908F4006A08F8
:10087600F5006B08F6006C08F700F001F101F201D3
:10088600F3016923013003180030F00070080319E2
:10089600842C83120030F4000030F5000030F6009E
:1008A6007F30F7006908F0006A08F1006B08F20073
:1008B6006C08F3006923013003180030F00070085B
:1008C6000319842C6908F0006A08F1006B08F2002D
:1008D6006C08F3000030F4000030F5002030F6001C
:1008E6008230F700D0217008E9007108EA0072082A
:1008F600EB007308EC0001308316A002031CA10371
:100906004C2C0030F4000030F5002030F600823028
:10091600F70083126908F0006A08F1006B08F2001C
:100926006C08F30069230130031C0030F0007008E6
:100936000319BB2C0030F4000030F5002030F6001F
:100946008230F7006908F0006A08F1006B08F200CF
:100956006C08F30031227008E9007108EA00720899
:10096600EB007308EC008316A00A0319A10A842C75
:1009760083162008A60721080318013EA7070130A1
:10098600A2000030A3000130F0000030F100E822A0
:1009960070088316A8007108A9007208AA007308D7
:1009A600AB0080302306F000803027067002031D5E
:1009B600DE2C260822020318FE2C0030F40000303C
:1009C600F5002030F6008230F7002808F0002908EC
:1009D600F1002A08F2002B08F30031227008831672
:1009E600A8007108A9007208AA007308AB00A20A41
:1009F6000319A30AD42C0030F4000030F5000030AF
:100A0600F6008030F7002808F0002908F1002A08CF
:100A1600F2002B08F30031226908F4006A08F50099
:100A26006B08F6006C08F70030217008E9007108C1
:100A3600EA007208EB007308EC000030F4000030A6
:100A4600F5002030F6008230F70069230130031CE0
:100A56000030F000700803193C2D0030E90000302A
:100A6600EA000030EB007F30EC008316A00A031981
:100A7600A10A831680302106F00080307002031D23
:100A8600462D003020020318812D83126D08840044
:100A960030308000ED0A6D0884002E308000ED0AAB
:100AA600803083162706F00080307002031D5D2D0E
:100AB600003026020318652D2608A002031CA10398
:100AC6002708A102FF30A200FF30A30080302106D4
:100AD600F000803023067002031D732D22082002C9
:100AE6000318812D83126D08840030308000ED0AD2
:100AF60001308316A202031CA303692DA201A301E0
:100B060080302306F000803027067002031D8D2DED
:100B1600260822020318F42D83126908F0006A08D9
:100B2600F1006B08F2006C08F3000C2370088316C2
:100B3600A4007108A5003030F00783126D08840008
:100B460070088000ED0A831623082106031DAD2DCB
:100B560020082206031DB52D83126D0884002E3051
:100B66008000ED0A83162408F0002508F100E8222B
:100B760070088316A8007108A9007208AA007308F5
:100B8600AB007008F4007108F5007208F6007308EF
:100B9600F70083126908F0006A08F1006B08F2009A
:100BA6006C08F30006237008E9007108EA00720871
:100BB600EB007308EC000030F4000030F500203044
:100BC600F6008230F700D0217008E9007108EA00CB
:100BD6007208EB007308EC008316A20A0319A30A35
:100BE600832D83126D08840080016F08F0000800D1
:100BF600243083120313FD00FD0BFF2D00000800B7
:0E0C0600831203133E088A003D088200080096
:100C140083120313BF01D0015F08E9006008EA00F2
:100C24006108EB006208EC003F30ED000330EE0099
:100C3400EB233F30E900D52370080A3CE700710834
:100C4400031C013EE801E80200306406031D2C2E5B
:100C540001306306031D322E80308316AD00D6208A
:100C640000306406031D382E02306306031D3E2E39
:100C7400C0308316AD00D62000306406031D442E18
:100C840003306306031D4A2E94308316AD00D6202C
:100C940000306406031D502E04306306031D562ED7
:100CA400D4308316AD00D620E501E601E501E60166
:100CB40080306606F000803068067002031D642EE2
:100CC4006708650203186E2E20308316AC00B92322
:100CD400E50A0319E60A5A2E3F30E900C223203000
:100CE4008316AC00B92356308316AC00B9236F3099
:100CF4008316AC00B9236C308316AC00B92374306E
:080D04008316AC00B9230800BE
:100D0C00831203137008F8007108F000F101F2016E
:100D1C00F301FB01FC019630F300FA017008F100BD
:0C0D2C007808F000F801F2012D2008000A
:100D3800C730831203139F052108F000F00D7010CF
:100D4800F00D7010F00D701070089F04FB251F1532
:100D58001F1DB02E0000AC2E1E08F100F0018316F6
:0A0D68001E08F0040030F10408003A
:100D72009C3083120313BA000630BB002130BC0042
:100D820000309F01C0309F0483161F179F178312E4
:040D92001F14080022
:100D9600831203135F08F1006008F2006108F30094
:100DA6006208F4000130DF02031CE002031CE102CA
:100DB600031CE2027408003C031DEB2E7308003C82
:100DC600031DEB2E7208003C031DEB2E7108003C40
:080DD6000318EE2ECB2E0800DD
:100DDE0083160313851085110610861006118611D1
:100DEE008312851085118611061186100610B62005
:100DFE00B620B620861406148514C3208510B6209E
:100E0E008514C3208510B6208514C3208510B62006
:100E1E0006108514C3208510B6208514C3208510B6
:100E2E00861086158514C3208510B62086110614EB
:100E3E008514C320851006108514C3208510B62096
:100E4E008514C320851006148514C3208510B62082
:100E5E0006108514C32085108615061586140614F3
:0C0E6E008514C3208510B620391408003C
:100E7A00831203135F08F2007208F100F20A600895
:100E8A00F000E00A700884000008F000710884008D
:100E9A00700880007108840000080319552F412F3B
:060EAA005F08F0000800E3
:100EB00003268A110A128000840ABD0A0319BE0A99
:080EC000F003031D582F080088
:10100000313083120313A2003630A3004630A4000F
:101010003830A5003730A6003730A7002030A800B0
:101020003230A9003030AA004D30AB002030AC0087
:101030004130AD004430AE004330AF003030B0003E
:101040002030B100B2010E3083169F00F1308500D0
:101050000E309F00FF30870083120713831688012C
:10106000F03086008312860180308316810083125F
:10107000850188141030DF002730E0000030E100E7
:101080000030E2008A11CB268A15831203138816DA
:101090008A11EF268A1580308316AD008A11D6207A
:1010A0008A153F30DF002230E0008A113D278A1583
:1010B0003F30E9008A11C2238A158A11B9268A15A0
:1010C000881083120313A1018A119C268A157008C7
:1010D0008312B3007108B4008A1186268A15003085
:1010E000F4000030F5002030F6007730F7008A1168
:1010F000D0218A157008B5007108B6007208B700D3
:101100007308B8007008DF007108E0007208E100A1
:101110007308E2000230E3000030E4008A110A267E
:101120008A15023088065030DF00C330E0000030FE
:10113000E1000030E2008A11CB268A1561289F2841
:02400E003A3B3B
:00000001FF
